:100000000EC0A0C1189518951895E6C118951895B9
:1000100018951895189518951895189518958FE5B1
:100020008DBFC0E4E8E24E2E82E08EBFD2E0F2E067
:100030005F2EA89584B7082E877F84BF88E1992713
:1000400081BD91BDEEEFF1E0A0E6B0E088278D9391
:100050003197E9F76624BA9885B7836085BFBB9866
:1000600086E886B980E087B93E983F9A3C98BC9A6A
:1000700087E08093500080E080934C007CB57062F4
:100080007CBD7CB570647CBD70E07BBD7FEF7DBDC9
:1000900084E083BF80E08ABD12D885E090E0A3D6DB
:1000A000B1D612D818E729D810E027D81AED25D8EC
:1000B00012E223D819D8CAD6E2EDF4E0A2E6B0E005
:1000C000ED93FC9381E08093600088E08093610071
:1000D000882780936400E4E3F1E1FBD5E3E0F0E0FE
:1000E000FED5B4D6709167007F777093670081E08A
:1000F0008093680080E0809369007BB770647BBF69
:10010000789479B7726079BF84E083BF79B77460FF
:1001100079BF87E080BF379AEF93FF93E4ECF0E07C
:1001200059D6FF91EF9107B1007F036007B943D71C
:10013000ABE6B0E08D939C93ABE6B0E00D911C91E3
:10014000063752E0150708F00CC081E0809360008C
:1001500081E7809361008827809364008EE3C5D592
:100160004AC0ABE6B0E00D911C91083A52E0150789
:1001700008F00CC081E08093600081E7809361000B
:100180008827809364008DE3B0D535C0ABE6B0E03E
:100190000D911C91003D52E0150708F00CC081E064
:1001A0008093600081E780936100882780936400DA
:1001B0008CE39BD520C0ABE6B0E00D911C91083FCD
:1001C00052E0150708F00CC081E08093600081E7E1
:1001D000809361008827809364008BE386D50BC0F1
:1001E00081E08093600081E780936100882780939D
:1001F00064008AE37AD500E010E020E030E0A5EE6C
:10020000B0E00D931D932D933C9381E080936A00A1
:1002100000916A000E3110F009F022C0A5EEB0E0A6
:100220000D911D912D913C91AAE6B0E0AD90BB24BB
:10023000ABE6B0E0AA0CBB1CAA0DBB1D4D915C91B6
:1002400066277727C5D6A5EEB0E00D931D932D93B5
:100250003D93AAE6B0E08C918F5F8C9308F4D8CFE1
:1002600000E11EE020E030E0A5EEB0E04D915D91B0
:100270006D917C913BD5A5EEB0E00D931D932D9330
:100280003D93A5EEB0E00D911D912D913C914EE175
:1002900050E060E070E02FD5A5EEB0E04D935D93A7
:1002A0006D937D93A5EEB0E00D911D912D913C9144
:1002B0004EE450E060E070E01ED5A5EEB0E04D9356
:1002C0005D936D937D93A9EEB0E0E5EEF0E096D6F8
:1002D00081E2A9EEB0E0EED48D9388278C9382E280
:1002E000A9EEB0E0E7D48D9388278C9383E2A9EE42
:1002F000B0E0E0D48D9388278C9307E00F93A9EEAC
:10030000B0E0D7D6482F0F91041BAAE6B0E00C93BB
:1003100000916A00003010F009F001C006C0909111
:100320006A00A9EEB0E0C6D4BDD481E0809360003D
:1003300081E080936100882780936400A9EEB0E09B
:10034000C2D4EACE0F921F922F923F924F925F92A9
:100350007F92AF92BF920F931F932F933F934F9330
:100360005F936F937F938F939F93AF93BF93CF933D
:10037000DF93EF93FF938FB78F93A5E6B0E08BD415
:100380007AE07BBD70916700706870936700EF93AF
:10039000FF93E8E7F1E01ED5FF91EF9170E47ABF9B
:1003A0008F918FBFFF91EF91DF91CF91BF91AF916F
:1003B0009F918F917F916F915F914F913F912F917D
:1003C0001F910F91BF90AF907F905F904F903F90A3
:1003D0002F901F900F9018950F921F922F923F927F
:1003E0004F925F927F92AF92BF920F931F932F9382
:1003F0003F934F935F936F937F938F939F93AF93AD
:10040000BF93CF93DF93EF93FF938FB78F93A9E6BB
:10041000B0E08C918F5F8C93009169000A3709F0EE
:1004200026C0A5E6B0E08D919C91A8E6B0E0AD9025
:10043000BB24ABE6B0E0AA0CBB1CAA0DBB1D8D9380
:100440009C9380E08093690080E090E0A5E6B0E0B6
:100450008D939C93A8E6B0E08C918F5F8C93009174
:1004600068000F3109F003C081E080936800A7E6BF
:10047000B0E08C9187FB0EF00CC08BB58A958BBDDC
:100480000BB5003009F005C0709167007F7770935D
:1004900067008F918FBFFF91EF91DF91CF91BF9157
:1004A000AF919F918F917F916F915F914F913F910C
:1004B0002F911F910F91BF90AF907F905F904F90C1
:1004C0003F902F901F900F901895F894FFCFF894BD
:1004D000FFCF0410400000000000000000000000FA
:1004E000000000000000000000000000000000000C
:1004F00000000000000000000000000000000000FC
:1005000000000000000000000000000000000000EB
:1005100000000000000000000000000000000000DB
:1005200000000000000000000000000000000000CB
:1005300000000000000000F8F860C080C060F8F81B
:1005400000F8F880C060003F3F00000100003F3F1E
:10055000003F3F01060C000000000000000000000A
:10056000000000000000000000E0E060606060E06B
:10057000C00000000080301800FFFFC0C0C0C0FFF6
:100580007F0000E0FC1F1830003F3F00000000002B
:1005900000383F07000000000000000000000000DD
:1005A000000000000000F0700000000000000000EB
:1005B0000000000000000300F8F800000000F8F858
:1005C00000000000000000000103030303033F3F9D
:1005D000000000000000000000000000000000001B
:1005E000000000000000000007070707070787C793
:1005F000F7FF7F1F0F0000000080E0F0FC3E1F07A8
:10060000030000000000001C1F1F1F1D1C1C1C1CE1
:100610001C1C1C1C1C080000000000000000000046
:1006200000000000000000000707070707FFFFFFAA
:1006300007070707020000000000000000FFFFFF9F
:100640000000000000000000181C1C1C1C1F1F1FC5
:100650001C1C1C1C18000000000000000000000012
:10066000000000000000000000FFFFFF0707070771
:10067000070FFEFEFCF0000000FFFFFF383838389F
:100680001C1C0F0F07010000001F1F1F00000000AF
:10069000000000000000000000000000000000005A
:1006A000000000000000000000000000000000004A
:1006B000000000000000000000000000808080803A
:1006C0008000000000000000000000000F0F0F0F6E
:1006D0000F0000000000000000000000000000000B
:1006E0000000000000000000FFFFFF0707070707EA
:1006F0000FFEFEF800000000FFFFFF1C1C1C7CFE2C
:10070000FFE78301000000001F1F1F000000000022
:1007100003071F1F1C18000000000000000000005D
:100720000000000000000000FFFFFF0000000000CC
:100730000000FFFFFF000000FFFFFF0000000000BF
:100740000000FFFFFF000000030F1F1E383838387D
:100750001C1E0F0700000000C0E0C0C080FCFCFCB5
:1007600080C0C0C0000000000103E3FBFF39187F18
:10077000FBF3630301000000000000010000000023
:100780000100000000000000000000000000000068
:100790000000000000000000000000000000000059
:1007A00000000000000000000000000000FEFEFE4F
:1007B000000000000000000E0E0E0E0E0EFFFFFFE8
:1007C0000E0E0E0E0E0600000000000000070707C8
:1007D0000000000000000000000000000000000019
:1007E0000000000000000000000000000000000009
:1007F000000000000000000000000000C0C0C0C0F9
:10080000C00000000000000000000000C7FFFF7FE4
:100810001F000000000000000000000000000000B9
:100820000000000000000000008080808080808048
:1008300080808080000000000103030303030303A2
:10084000030303030000000000000000000000009C
:100850000000000000000000000000000000000098
:100860000000000000000000000000000000000088
:10087000000000000000000000000000C0C0C0C078
:10088000C00000000000000000000000070707078C
:100890000700000000000000000000000000000051
:1008A0000000000000000000000000000000000048
:1008B0000000000000000000000000000000000038
:1008C0000000000000000000000000000000000028
:1008D00000000000000000000080C0E0F07070F038
:1008E000E0C08000000000E0FEFFFF070000000005
:1008F00007FFFFFEE000003FFFFFFF0000000000D9
:1009000000FFFFFF3F000000030F3F7F787070780B
:100910007F3F0F03000000008080C0C0C0E0E0F017
:10092000F0000000000000000303030101FFFFFFCF
:10093000FF000000000000000000000000FFFFFFBB
:10094000FF0000000000000030303030303F3F3FFB
:100950003F30303030300000C0E0E070707070F038
:10096000E0E0C00000000000000000000000008087
:10097000FFFFFF7F00000000000080E0F0FC3E1F52
:100980000F030100000000003C3F3F3F3330303098
:10099000303030300000000000E0E0F0707070F0A7
:1009A000E0E0C0000000000000000000000080C087
:1009B000FFFF7F1F00000000000001030303070F7B
:1009C0003FFEFCF8E0000000003870707070707836
:1009D0003E3F1F0F03000000000000000000C0E0C9
:1009E000E0E0E000000000000000C0F0FC7F1FFF1E
:1009F000FFFFFF00000000F0FCFFFFE7E1E0E0FF89
:100A0000FFFFFFE0E0000000000000000000003FEA
:100A10003F3F3F000000000000E0E0E0E0E0E0E0F9
:100A2000E0E0E0E00000000000FFFFFFC0C0C08089
:100A30008000000000000000000101010101030727
:100A4000FFFFFEF80000000030707070707070786A
:100A50003F3F0F0700000000000080C0E0E0F070A2
:100A60007070F0E0C0000000F0FEFFFF87C1C0C062
:100A7000C0C0800000000000FFFFFFFF0701010170
:100A8000030FFFFFFCE00000010F1F3F7C70707040
:100A9000707C3F1F07010000E0E0E0E0E0E0E0E004
:100AA000E0E0E0E0E000000000000000000080E086
:100AB000FCFF1F0701000000000000C0F0FEFF1F48
:100AC000030000000000000000303E3F3F0F000028
:100AD00000000000000000000080C0E0F0707070B6
:100AE000F0E0E0C000000000003FFFFFF1E0C0C008
:100AF000F0FF7F1F00000000F0FCFE7F0F07070FD4
:100B00001FFEFCF8F0000000071F3F7E7870707039
:100B1000783F3F1F070000000080C0E0F07070F0D9
:100B2000E0E0C00000000000FEFFFF8300000000C6
:100B300001FFFFFFFC00000001070F1F1E1C1C1C13
:100B40000EFFFFFFFF0000000038707070707078BB
:100B50003E1F0F07000000000000FF81BDBDBDBDAE
:100B6000BDBDBDBDC33C0000000000000000000092
:100B70000000000000000000000000000000000075
:100B80000000000000000000000000000000000065
:100B900000000000000000000000FF81BDBDBDBDE1
:100BA000BDBD8181C33C00000000000000000000CA
:100BB0000000000000000000000000000000000035
:100BC0000000000000000000000000000000000025
:100BD00000000000000000000000FF81BDBDBDBDA1
:100BE00081818181C33C0000000000000000000002
:100BF00000000000000000000000000000000000F5
:100C000000000000000000000000000000000000E4
:100C100000000000000000000000FF81BDBD8181D8
:100C200081818181C33C00000000000000000000C1
:100C300000000000000000000000000000000000B4
:100C400000000000000000000000000000000000A4
:100C500000000000000000000000FF818181818110
:100C600081818181C33C0000000000000000000081
:100C70000000000000000000000000000000000074
:100C80000000000000000000000000000000000064
:100C9000000000000000ED91FC91EF5FFF4FFC931E
:100CA000EE93089580E2903019F08D939A95E9F7CC
:100CB0009C9308958F938D918823E9F711978F91D5
:100CC0000895A0E1B2E08D91882311F00ED0FBCF02
:100CD00008957AD1802D11F008D0FBCF089588EEC9
:100CE00093E081D03197D9F70895BCC050D00AD095
:100CF00000FC05D008954BD020D001F8F9CF52D098
:100D00005AD00895842F952FA62FB72F4427552703
:100D100066277727F1E2889409C020F4480F591F0D
:100D20006A1F7B1F76956795579547953795279549
:100D300017950795FA9589F70895842F952FA62F73
:100D4000B72FE894452B462B472B11F46894089550
:100D5000402F512F622F732F00271127222733276F
:100D6000F0E2440F551F661F771F001F111F221F3F
:100D7000331F081B190B2A0B3B0B416028F4080F8B
:100D8000191F2A1F3B1F4E7FFA9559F7089500241B
:100D9000E89477FF02C006D0689400F809D010F8F4
:100DA0000124089512D04F5F5F4F6F4F7F4F08951A
:100DB000E89437FF089500951095209530950F5FC2
:100DC0001F4F2F4F3F4F6894089540955095609561
:100DD000709508953197F1F70895689462F8089531
:100DE000E89462F80895EF93FF93EE27E82BE92B40
:100DF00031F0E0EDF7E03197F1F70197D1F7FF918E
:100E0000EF91089561D1E8E1FEE05AE1DDD0102DC7
:100E100074D15A95D9F768C178AED580003FD30018
:100E2000408D142000A1C8DA1281FFD9F1D840A466
:100E3000A6AF4AD118E761D1182F06C018E744D1F0
:100E40005CD110E45AD1182F58D14EC13DD118E7CA
:100E500054D110E452D11127E0E0F4E04ED13197A3
:100E6000E9F742C1EF93FF93509160005F93709058
:100E70006100E0916200F0916300A6D0202DA4D023
:100E8000302DA2D0002DA0D0602D8052482F05D14A
:100E9000E40FF51FCC241124E22E603051F1DD2443
:100EA000DA94CD2CFF24032F8FD021F00A95E00F88
:100EB000F11D03C0F3940A95B9F7FD1408F4DF2C73
:100EC000EA9481F7E22EFF24032F3197C895002082
:100ED00021F00A95E01BF10903C0F3940A95A9F7E4
:100EE000FC1408F4CF2CEA9471F7D31611F4D62E23
:100EF000CC2470926100732F7C1940916100509155
:100F000060003FD0603039F0DD2029F05D2D5CD0ED
:100F10005A95E9F77D1958D0802D509164005523DA
:100F200009F080958BDF50916100539550936100DB
:100F30007A9589F7EC0DF11D603079F050916400DD
:100F4000762F8827552309F0809578DF7A95C9F7A1
:100F500050916100560F509361005091600053957D
:100F6000509360002A9509F0C4CF5F9150936000C0
:100F7000FF91EF91089507D0A7D018E7BED010E4F5
:100F8000BCC04A955A954F939FD018E7B6D010E051
:100F9000B4D010EB150FB1D01F911F9312951F7095
:100FA0001061ABD01F911F70A8D09EC0019111910C
:100FB000219130810895369A3699FECF369A369926
:100FC000FECF84B195B10895C8953196002008955B
:100FD000040F151F261F371F0895000F111F221F12
:100FE000331F089500951095209530950F5F1F4F82
:100FF0002F4F3F4F0895019110810BC0D7DF0BC0D9
:101000000191108117FF05C03FEF2FEF04C0008151
:1010100011272227332737FF03C0E4DF8DE28D93AA
:10102000CF92DF92EF92AA24BB24CC24DD24EE24BD
:1010300040E2EAE0FF2755E093E38081890F87FDD6
:101040009F7083FD907F891B81935A95A9F7C5DF17
:10105000AA1CBB1CCC1CDD1CEE1C4A9551F7E89465
:10106000EFE0FF2782910CD0EB30E0F71EF06894A0
:101070008A2D0AD088278D93EF90DF90CF90089526
:10108000982F829501D0892F8F70805D26F0803354
:1010900009F4089568948D930895FF935527F8E017
:1010A000469508F4500F57954795FA95D1F7FF915B
:1010B00008958FEF83959D919923E1F70895B9984D
:1010C000B898C198C0980895B89AB99803D0B898BC
:1010D00001D0B99A000000000000000000000000EC
:1010E0000000000000000895B89AB99AF3DFB8989C
:1010F000B09BFECFEFDFB998EDCF0894111F01C070
:10110000110F69F0B89A18F40000B99802C0B99AA2
:1011100000C0E0DFB898B09BFECFDCDFF1CFB89A1B
:10112000B998D8DFB898B09BFECFE894B19968948D
:0C11300062F8D0CF39242526272829009A
:00000001FF
